:020000040800F2
:10500000981A0020D5500008F1820008197B00088A
:105010000000000000000000000000000000000090
:105020000000000000000000000000009D9000084B
:10503000000000000000000049890008B991000844
:10504000E7500008E7500008E7500008E750000864
:10505000E7500008295B0008E7500008E750000807
:1050600000000000E7500008515A0008E75000080F
:10507000E75000086D7F000800000000E7500008BE
:1050800000000000E75000080000000000000000E1
:10509000E750000800000000E7500008E750000853
:1050A000E7500008E7500008E7500008459900085D
:1050B000E7500008E7500008000000000000000072
:1050C0000348854600F060FC0048004771A70008CF
:1050D000981A00200448804704480047FEE7FEE78E
:1050E000FEE7FEE7FEE7FEE755920008C150000824
:1050F00030B50B46014600202022012409E00D4670
:10510000D5409D4205D31D469540491B25469540F7
:1051100040191546521E002DF1DC30BDF0B51FB40C
:105120000646002082B005464024019100901BE015
:10513000019922460F46304600F04EFB049A059B2B
:10514000801A994110D310461946224600F034FBCC
:10515000361A8F410197224601200021009F00F05E
:105160002BFB38184D4100902046641E0028DFDCE0
:10517000019B00982946324607B0F0BD03460B4319
:105180009B0703D009E008C9121F08C0042AFAD2FD
:1051900003E00B780370401C491C521EF9D2704783
:1051A000D2B201E00270401C491EFBD270470022BF
:1051B000F6E710B513460A4604461946FFF7F0FF16
:1051C000204610BD30B504460020034600E05B1CBD
:1051D000934203D2E05CCD5C401BF8D030BDF8B503
:1051E00002464A40D40F42004B0052085B089A42E4
:1051F00002D20246084611464A0023D0C30D4A0097
:10520000DDB2120EAD1A202D35DA49020126490A07
:10521000F6058A19002C00D0524220214F1B11465E
:10522000B9402A411018C20D9A4221D0002C17D043
:10523000012D08DCDA05801AD20F8019D207DBB203
:1052400000F0F6FAF8BDDA05801A012340001B06CB
:10525000C01880185A428018CA0F1043490007E04E
:105260004908C2071143DA05801A801940088018DE
:1052700000F0D6FAF8BD61000122511A001BF7E7D1
:105280000122D2075140AAE70122D2075040A6E7E7
:1052900070B502464A40D50F40004A00ED0740086D
:1052A0005208002814D0002A12D0C40DD30D410298
:1052B0000120C0055202490A520AE41A09181218BC
:1052C0007D34914201D3641C00E04900002C01DAD6
:1052D000002070BD0023914201D3891A0343400886
:1052E00049000028F7D100290AD0914202D10121BA
:1052F000C90705E0914201D2012101E00121C94322
:10530000E005C018401900F08BFA70BDF0B50746F3
:105310000846584087B0C00F049048000E46590018
:1053200040084908BC1A884105D2384631461E4615
:1053300017460B4602465800400810434CD0300D2B
:10534000039040055900400D490D0590401A029008
:10535000402872DA18030121000B09050843019067
:1053600004980092002805D00199524200208841FB
:1053700000920190029840210A1A0199009800F0C9
:105380001BFA05460C466B4607CB00F036FAC019EF
:105390007141039A0E0D0023D71756401A467A40E2
:1053A000164344D0049A002A2DD0029A012A039A67
:1053B00015DC1205C01A914101263605001C714109
:1053C000D20F059ED2070093019202962A462346E9
:1053D00000F074FA07B0F0BD38463146FAE716051A
:1053E000224A0F46B218C01AB74101210905001C14
:1053F0004F4100187F41114618187941E20F1043C0
:105400006D19644113E0E2076D0815436408C20793
:105410001443039A01261205C01A91413605001C57
:105420007141CE07400830434908C01851412A460F
:10543000234600F036FACDE7FFE70498012240004A
:10544000C117121A00238B4104983146C417381A29
:10545000A141EEE730B40124E407634030BC55E7D6
:1054600030B40124E407614030BC4FE70000E0FFA6
:10547000F0B51FB488B00B990998002448400999E9
:10548000C00F490049080991C0070B9900904900D5
:1054900049080B9109990898A64608431CD00B9916
:1054A0000A98084318D0099801244000420D48008A
:1054B000410D099824050003000B204309900B9827
:1054C0000003000B20430B9050181C494018002289
:1054D00001901446104605E0002001460DB0F0BDD5
:1054E000032801DA034600E003239C46C11A0AAEF2
:1054F0000AE05F0008ADED5B4F00F75B7D430027DE
:10550000AA187C41491C5B1E6145F2DD410004ABD9
:105510005A522104120C0A43240C401C0828DFDBD9
:10552000019802900099704601910090059B049AA1
:105530000799069800F0C2F9D0E700000DFCFFFFC4
:10554000F0B50C465C4085B0E40FE40703944C00D2
:1055500000266408590094464908024602962243F0
:1055600021D062460A431ED06200570D4A000E0346
:105570002303550D012402462C492405781B1B0BDF
:10558000360B401823432643614600901C46501AB0
:10559000B44103D30098401C009002E09218009898
:1055A0005B41002803DA0020014605B0F0BD002071
:1055B000012109050746864611E064461D46141B75
:1055C000B54106D36546521BB341744607430C43AD
:1055D000A646CD0740084908284392185B41054676
:1055E0000D43EAD11046184313D060461946504087
:1055F0007140084306D06046101AB34106D201221A
:10560000002306E000220123DB0702E00122D2434F
:105610005310009874460105381C6141029C039D9B
:105620000019694100F03DF9BFE70000FD030000EB
:10563000C217C10F504010B54018CA079623002169
:1056400000F0F6F810BD10B500229623114600F0C8
:10565000EFF810BD0EB5C217C10F5040CA07401871
:105660000021054B0293019200910A460B4600F07F
:1056700025F903B000BD0000330400000EB5054954
:105680000291002100910A460B46019100F016F9A3
:1056900003B000BD33040000410040020122400A73
:1056A000D205090E80187F2901DA0020704796295B
:1056B00003DC9622511AC8407047963988407047DB
:1056C00070B5CD0F4A0009030123090B1B051943CF
:1056D0000B4BED070024520D9A4201DA002070BDF9
:1056E000074B34339A4203DC9A1A00F075F802E053
:1056F0000449511888402C43F1D0404270BD00004D
:10570000FF030000CDFBFFFF4A0009030123090B43
:105710001B051943094B10B5520D9A4201DA0020BE
:1057200010BD064B34339A4203DC9A1A00F054F849
:1057300010BD03495118884010BD0000FF03000050
:10574000CDFBFFFFC20FD207400040080BD0C10DB8
:105750000723DB01C91840020905400A1143C208AA
:10576000400711437047002001467047CB0FDB070D
:10577000490010B5490802460A4307D00A0D07241C
:105780000903E401090B121B002A01DC002010BDF3
:10579000C900440F0C43C100E018D205801800F086
:1057A0003FF810BD0122D207002800DB101A0029A3
:1057B00000DB511A8142704710B5202A04DB0146F4
:1057C000203A9140002010BD914020239C1A0346AE
:1057D000E3401943904010BD10B5202A04DB084671
:1057E000203AD040002110BD0B46D340D0402024A9
:1057F000A21A91400843194610BD10B5202A06DBB5
:10580000CB170846203A1041C1170B4306E00B4660
:105810001341D0402024A21A91400843194610BDDC
:10582000002904DA401C490001D1400840007047BB
:1058300070B40024050C05D11024000402D1002905
:1058400021D01124050E01D100020834050F01D129
:105850000001241D850F01D18000A41C002801DB5C
:105860004000641C002908D020252E1B0D46F54061
:10587000A14000D001212943084301061B1B000A57
:10588000DB1D02D5002070BC7047DB05181880189E
:105890000029F8DA401C4900F5D170BC40084000EE
:1058A000704710B5002B08DA0024401C61419218A3
:1058B0005B411A4301D14008400010BDF0B51FB450
:1058C00082B005460C0003D0084604F0FBF802E065
:1058D00004F0F8F820300246009021462846FFF7F1
:1058E0006BFF049B059A04460F4618431143084377
:1058F00014D0184610431BD0009840210A1A1846AD
:105900000599FFF769FF05460E46009A0599049828
:10591000FFF752FF084305D0012004E02046394636
:1059200007B0F0BD0020C11705430E432C43374399
:1059300000990E986305401A7905E40A00220C4389
:10594000FD0A0A3002D500200146E9E701051019D9
:1059500069410C9C0D9D00196941FFF7A2FFDFE72B
:1059600010B5002904DB0124E40740428C412146A4
:10597000002B04DB1C460123DB075242A341994262
:1059800000D1904210BD0000064C0125064E05E0F6
:10599000E36807CC2B430C3C98471034B442F7D350
:1059A000FFF792FBE4AA000804AB000838B50446F0
:1059B000064805490068FFF79BFB604300E0401E76
:1059C00000900028FBD138BD40420F001C01002090
:1059D000F8B50446006881688907890F012902D15A
:1059E0000168C90722D18168114A1026114001259A
:1059F00000290ED18168294381600120FFF7D6FF7D
:105A000000F07AFF07460CE000F076FFC01B0A2882
:105A100007D9606D30436065A06D2843A065012003
:105A2000F8BD20680068C043C007EDD10020F8BD74
:105A30001700008010B500231A4603E0845CE318C9
:105A40009BB2521C8A42F9D3D84380B210BD0000E9
:105A500010B5034800F010FD024800F00DFD10BD28
:105A600038160020F015002030B5446C1C252C4061
:105A70000125A540046C6560046863608368102B91
:105A8000036803D099600068C26030BD9A60006806
:105A9000C16030BD1449012048720A4602205E32BE
:105AA000507203203C3A507204200E3A50720F4854
:105AB0000D4B0078087022310870203108770C49AE
:105AC0005A1C0878587149789971233318715971A3
:105AD000203318775977107551751A461E32107594
:105AE000517510765176704750110020D700002074
:105AF000F400002010B503F0A9FA202003F052FBB7
:105B0000012004F08FFB002003F04CFB044804F05C
:105B10002DFA044804F0DCFC002004F011FD10BD57
:105B2000C000002083800000F8B505200121000797
:105B300000F0D2FE0025184C002800D06560174EFA
:105B40000221304600F0C8FE00281DD1012020703F
:105B50001348808F00280ED00127BF02002239464B
:105B6000304600F0C2FE0A2004F0B2F901223946A4
:105B7000304600F0BAFE0B48656000880A214843B1
:105B80000949088003F0F0FE012000F0DDFD02204D
:105B900000F0DAFDF8BD00000C0100200004005008
:105BA000500D0020E4000020F000002070470000AD
:105BB00010B5084900224A6107494B684C15234338
:105BC0004B604B68082423434B60C009C00102604E
:105BD00010BD000080160020002002407FB5002587
:105BE0000C460646039500F07FFDE009029003A9EC
:105BF00001960095684600F00FFD002804D000F0E3
:105C000047FD002004B070BD00F042FD0120F9E71F
:105C100010B5002302E0C45CCC545B1C9342FAD361
:105C200010BD000010B5214A00219069C30520482D
:105C300004D54169022319434161911593699B057C
:105C400005D54369012423434361630219439369E2
:105C50005B0505D54369082423434361E3011943E8
:105C600093691B0505D543690424234343616302FB
:105C7000194393699B0405D5436910242343436169
:105C80006302194393699B0304D5446920231C4391
:105C9000446119439369DB0305D5436940242343D9
:105CA0004361A0020143916110BD00000020024049
:105CB0008016002070B5054600F01EFE0646184C02
:105CC0000AE0681C08D0002D04D000F015FE801BEF
:105CD000A84201D9032070BDA069C007F1D1A06915
:105CE000800701D50220A061A069C00511D4A06978
:105CF00080050ED4A06940050BD4A069000508D426
:105D0000A069800405D4A069800302D4A069C003FF
:105D100003D5FFF787FF012070BD002070BD000094
:105D200000200240F8B51746002605460C4600F054
:105D3000DBFC09E029460220226800F0B7FC0028BD
:105D400004D1241D2D1D361DBE42F3D300F0A0FC4E
:105D5000BE4201D20020F8BD0120F8BD10B50849AF
:105D600002460020054B497905E044001C5B944243
:105D700003D0401CC0B28842F7D310BD7812002077
:105D80005800002010B500F0ACFD10BD10B509485A
:105D900000F0D4FF80B2FFF771FC074A074BFFF712
:105DA00067FB0022064BFFF7CBFBFFF7ADFC80B291
:105DB00010BD0000E8140020F853E3A59B843E408A
:105DC00000408F4070B5324930488A7F0275C97FE4
:105DD000417530490A780276497841762B49052089
:105DE000133148720A2004F063FB7D20C00004F0E8
:105DF00079FB2649002213310C2004F043FC0021DA
:105E00000C2004F051FC022004F0A2FB224C204D97
:105E100000210F2004F0CCFA20422863F8D0286B30
:105E2000411C30D040042DD58122D20100210F2009
:105E300004F0FDFB0021102004F0BAFA41061348DB
:105E4000490E0022633004F0E9FA104C6334607AA2
:105E5000052817D102220F49601DFFF7B3F900286A
:105E600010D10B48A67C6E710422611C4430FFF7F0
:105E700085F921461331084672005130FFF77EF94B
:105E80000320287070BD02F057FA0000B111002005
:105E900058000020F400002000D0272410B5084846
:105EA00000F096FA0A21064800F032FA044800F0A1
:105EB0001DF9800503D5024800F01AF980B210BD23
:105EC0008C140020F8B52F4D00220121284600F047
:105ED0000CFDFFF7E3FFFFF7B6FB2B4E3146FFF754
:105EE000D7F92A4C0122A0601146284600F0FDFC9B
:105EF0002749A068002588423EDB2078254F0028EE
:105F000015D02570FFF7CAFFFFF79DFB3146FFF75D
:105F1000BFF9A060FFF716FC00223B46FFF79AFA94
:105F200000221D4BFFF7A4FAFFF720FC6060A06879
:105F3000FFF708FC00223B46FFF78CFA174A184B84
:105F4000FFF796FA06460F466068FFF7FBFB134A19
:105F5000144B5242FFF78CFA32463B46FFF7D6F914
:105F6000FFF704FC10496060884201DD616004E0D5
:105F7000FF21C905C84200D365606068FFF78CFB4C
:105F8000C0B2F8BD0004005000401B4430000020A7
:105F90000000604000000C4000E0644033333333C5
:105FA00033B33040CCCCEC3F0000C842F8B50546D6
:105FB00004464035287C0026012808D0012028749A
:105FC000206881688907890F01290ED101E002202C
:105FD000F8BD0168C90708D0606D202108436065DD
:105FE0000126002028743046F8BD616DFF22013281
:105FF0009143022211436165C1688907890F0091AD
:10600000C16889088900C1602068816892071143CE
:10601000816000F071FC07460EE000F06DFCC01BD3
:106020000A2809D9606D0221884310210843606560
:10603000002028740120F8BD206880680028ECDB6F
:106040002068C168009A1143C160606D80088000BB
:10605000401C6065C5E70000F8B506460D464036B1
:10606000317C01290DD00121317401688A68520701
:1060700009D5416D20221143416500203074012073
:10608000F8BD0220F8BD174B6A68D80547109A4240
:10609000154C8A6A2B6812D05B035B0B1A438A6229
:1060A0002968490305D5A1680143A1600A20FFF7CB
:1060B0007DFC2868800312D5A06838430EE05B039E
:1060C0005B0B9A438A622968490302D5A168814320
:1060D000A1602868800302D5A068B843A0600020B2
:1060E0003074F8BD0110000000270140406D70477A
:1060F0000068006C7047000070B5040006D0606D49
:10610000264600254036002802D006E0012070BD5A
:10611000A5653574204600F0D3F8606DC00603D441
:1061200021688868400705D5606D102108436065C7
:106130003574EBE7606DFF22013290430222104379
:10614000606588688207920F5B48012A02D10A685D
:10615000D2072BD1032362689B079A4205D05B428A
:106160009A4202D05B009A4209D10A6992009208D1
:106170000A6121680A6963681A430A610CE00A69C6
:10618000920092080A6181680F2292049143816013
:1061900081686268114381602168CA6818239A4344
:1061A000CA602168CA68A3681A43CA60816801226C
:1061B0005206914381608168A28E5206114381602C
:1061C00020688168C90004D4816801221207114344
:1061D00081602068C168394A1140C1602069E16866
:1061E000022825D000200143204620300278037B7E
:1061F00052035B001A431143226B1143A2699203BD
:106200001143E269D20311432268D3681943D16074
:10621000616A0A46FF3AC23A05D0A26A114322686F
:10622000D3681943D16042780121012A02D00BE0E2
:106230000420D8E70078002823D0606D2022104386
:106240006065A06D0843A065E06B012820681FD041
:106250000169C90703D00169490849000161206843
:106260004169C908C900416120684169A26B1143B5
:106270004161A565606D80088000401C606500205C
:1062800070BD2068C26801231B041A43C260DBE7AB
:106290000269FF239B009A43026120680269236C14
:1062A000A66C1A43636C33431A4302612068026987
:1062B0000A430261D3E70000002701401902FEFFF4
:1062C00010B586B0044614216846FEF770FF0E49EB
:1062D0002068884216D10D48416B42151143416335
:1062E000C16A01221143C162C06A6946104005902B
:1062F000022000900320019000200290052000075A
:1063000000F02EFA06B010BD00240140001002403B
:10631000F8B504464069254640350E4608280BD09E
:106320002068C068C00709D0606D202108436065FF
:10633000002028740120F8BD082700E00C2700F099
:10634000DBFA009011E0701C0FD0002E05D000F099
:10635000D3FA0099401AB04207D9606D042108436E
:106360006065002028740320F8BD2068006838426A
:10637000E9D0606D01214902084360652068C16869
:1063800009058A0F0C21002A1BD12022125D002A48
:1063900017D10268120714D5826853070122002B17
:1063A00008DB43688B434360606D130298431043DE
:1063B000606506E0606D202318436065A06D1043A2
:1063C000A065A069002801D1206801600020F8BD07
:1063D00070B50446216800208968490721D4254604
:1063E0004035297C01291CD001212974E16901294A
:1063F00004D02046FFF7ECFA002811D1616D0A4A5B
:106400001140FF220132114361650021A165297409
:1064100022681C21116021688A6804231A438A605B
:1064200070BD022070BD0000FEF1FFFF70B50024BA
:10643000014620314A79022A03D00421C163012494
:1064400018E0026813680E25AB43136002681368F6
:106450005B085B001360436C1C221340012215464D
:106460009D40036C5D604A7100220A71816B0029B6
:1064700000D08847204670BDF0B4016C0D680168FB
:106480000C68466C1C2304221E401746B7402F425E
:106490000ED067070CD50C68A40602D40C68944390
:1064A0000C60416C19408A40016C4A60016B1AE033
:1064B0000227B74002462F402032002F17D0A707EF
:1064C00015D50C68A40605D40C680A25AC430C60ED
:1064D00001215171446C02211C40036CA1405960A0
:1064E00000211171C16A002918D0F0BC08470827A3
:1064F000B7402F4212D0240710D50C680E25AC43AC
:106500000C60446C01211C400B46A340046C63608A
:10651000C163517100211171416BE4E7F0BC704718
:1065200070B504003CD01F48256814212818FEF7D8
:10653000DFFD800060641C4820640221204620307A
:106540000246417129681948E3680140A0686669FC
:106550001843236933431843A3691843E369184375
:10656000236A1843084328600121A06889038842F0
:1065700010D00D488030836A656C1C210D400F26B9
:10658000AE40B3438362656C63680D40816AAB4083
:106590000B4383620020E06301215171107170BDD3
:1065A000012070BDF8FFFDBF000002400F80FFFF1B
:1065B000F8B504468C46203001790025012909D020
:1065C0000126067141790027012905D007710225AE
:1065D0002846F8BD0220F8BD02214171E76320681A
:1065E000016849084900016061462046FFF73CFA0E
:1065F000206B00282068016801D00E2205E00422EB
:1066000091430160206801680A22114301602068FB
:10661000016831430160DBE7F8B51A4E0546307C6E
:106620000F46012807D0012030741748FFF742FBBE
:10663000010002D021E00220F8BD0020C0433860F4
:106640006C6814E02046FFF7B3FA0F48FFF732FBFF
:1066500001460E48426808239A4342604268431547
:106660009A434260002901D03C6006E08034A8686B
:106670006A68C0018018A042E4D80020307408463F
:10668000F8BD00008016002050C30000002002402A
:1066900005484168022211434160416801221143CB
:1066A000416000207047000000200240F8B50C4C0B
:1066B0001646207C0F46012808D001202074094886
:1066C000FFF7F8FA0025002802D006E00220F8BD06
:1066D00065613E600348FFF7EDFA2574F8BD0000E0
:1066E0008016002050C3000011484168C9070BD034
:1066F000EFF3108172B60F4AC2600F4AC26081F395
:1067000010884168C9070ED1416889070DD5EFF39C
:10671000108172B6094A0261094A026181F3108848
:106720004068800701D501207047002070470000B5
:1067300000200240EFCDAB8905040302BFAE9D8C63
:10674000161514137047000010B504494A69024237
:1067500002D04861FFF7F6FF10BD000000040140C1
:10676000F8B500230124A2E027469F403A4070D0AC
:106770004D68022D01D0122D14D1DD08AD002D1869
:1067800000952D6A5E07AC46F50E0F26AE46AE406C
:106790006546B543AC460E697546AE4065462E4328
:1067A000009D2E624D68012D05D0022D03D0112DC4
:1067B00001D0122D16D185680326AC465D00AE4689
:1067C000AE406546B543AC46CE687546AE406546BC
:1067D0002E43866046680D79BE43ED06ED0F9D4061
:1067E0003543456006685F000325BD40AE46AE43B5
:1067F0000D79B446AE07B60FBE4065462E4306601F
:10680000C6687546AE438D68BD403543C5604D686A
:10681000ED004BD5294D6E6B26436E639E08284DC7
:10682000B6007519AC46AD689E07360F0F27B74006
:10683000BD4305273F07B84201D1002715E0214F8E
:10684000B84201D1012710E01F4FB84202D1022700
:106850000BE02BE01D4FB84201D1032705E01C4F90
:10686000B84201D1052700E00627B7402F4365460F
:10687000AF60184D2E684F689643FF0300D516434E
:106880002E606E684F689643BF0300D516436E6056
:10689000AE684F689643FF0200D51643AE60EE68BF
:1068A0004F689643BF0200D51643EE605B1C0A6832
:1068B0001546DD4000D057E7F8BD0000001002404B
:1068C000000001400004005000080050000C00507F
:1068D000001C0050000401400069084000D0012065
:1068E000704742694A4042617047002A01D0816185
:1068F00070478162704700000148006870470000DF
:106900001801002002480168491C0160704700001E
:106910001801002010B508480024016840221143E6
:106920000160204600F00AF8002801D0012401E0AF
:1069300000F030FA204610BD0020024070B5054638
:1069400009487D210024C9000068FEF7D1FB00F052
:10695000C5FE002801D0012404E000222946501E73
:1069600000F038FA204670BD1C01002070477047C7
:10697000F8B5664CA078401CA07001202071E08A18
:10698000401CE0826248008802F0C6FB6148C08873
:10699000FEF759FE6049FEF77BFC604D2968FEF763
:1069A0001EFC28606078002500280BD102215C487D
:1069B000FFF792FF02005B495B4819D00022FFF706
:1069C00094FF2563594E01203768C005874257DB85
:1069D000208AFEF738FE01467F20C005FEF758FCEE
:1069E0003946FEF751FC306051480221017049E000
:1069F0000122D1034C48FFF778FF4648C088FEF7D4
:106A000022FE4549FEF744FC216BFEF7E8FB4949AD
:106A100020638842D6DD3F480127F92640300090A8
:106A20000A213046FEF764FB002903D13D493E4868
:106A3000FFF7A8F902213A48FFF74EFF002801D0DE
:106A4000002701E0002F12D102213548FFF744FF53
:106A500000280CD103F056FF00990120888003F034
:106A6000B1FF642003F034FA34493348C8600A2087
:106A700003F02EFA3046761EF6B20028D0D1A1E7F8
:106A80002B48057002212648FFF726FF002809D071
:106A90002563224E2A4937682A488F4214DD012196
:106AA000017012E01B48C088FEF7CDFD1A49FEF7C1
:106AB000EFFB216BFEF793FB234920638842E8DB61
:106AC0001E491D48C860E4E705701248408F401E0B
:106AD000FEF7AEFD3946FEF765FE06D86079002860
:106AE00003D01A490120087001E0184805700948D0
:106AF000408FFEF7A8FD3168FEF754FE04D260799E
:106B0000002801D003F0C2FEF8BD0000D400002030
:106B100074000020500D002000007A441001002075
:106B2000000400500080000000000050140100200C
:106B30006B000020000040400400FA0500ED00E07A
:106B40000000F0425E0000200000A0406D00002028
:106B5000704770B505000DD002202C462034A0737C
:106B6000284601F00BFA284600F0BEF80020A0737A
:106B7000607370BD012070BD7047704710B504464A
:106B800000680168C943C90708D18168C943C907BA
:106B900004D1012141602046FFF7EAFE2068016828
:106BA000C943890708D48168C943890704D40221ED
:106BB00041602046FFF7DAFE20680168C9434907B3
:106BC00008D48168C943490704D4042141602046A0
:106BD00000F0DEF820680168C943090708D481681D
:106BE000C943090704D4082141602046FFF7B0FFDC
:106BF00020680168C943C90608D48168C943C90629
:106C000004D4102141602046FFF7B1FE20680168DE
:106C1000C943890608D48168C943890604D4202160
:106C200041602046FFF7A9FF20680168C943490673
:106C300008D48168C943490604D4402141602046F4
:106C4000FFF79AFF10BD0000F8B5040005D02546F7
:106C50002035A87B002802D006E00120F8BD0020E6
:106C60006873204600F052F80220A8732068C268BA
:106C700084466368012B04D00120A16AC0058142CB
:106C800001D11E20824315486169814201D0144818
:106C900002401448A668024018463043676A266AD4
:106CA0003E433043A66A30431043012B03D00122F8
:106CB000D205964203D12369E2681A431043074A7A
:106CC000914205D0A2691143E2690243084610438C
:106CD0006146C8600120A8730020F8BDFFFF0000D6
:106CE0003F1FFFFFF8F119FF10B500680549884202
:106CF00007D10548816B4900490881630D2000F0E8
:106D000055F810BD007C00400010024010B500682E
:106D1000084988420CD10848816BC2041143816341
:106D2000002201210D2000F055F80D2000F048F858
:106D300010BD0000007C0040001002400068C069E7
:106D40007047000070B50224034620339C730F4C3B
:106D50002568E604354325600468E568B6123543C6
:106D6000E5600568AE6801242643AE6005682E69BB
:106D700026432E610568A96101684A6100680169BE
:106D80000422114301619C73002070BD0004014086
:106D9000704700000448416B012211434163816B3D
:106DA000020411438163704700100240C106C90EFE
:106DB00001208840014908607047000080E100E040
:106DC000C106C90E012088400149086070470000D3
:106DD00000E100E010B501F08DFA10BD02494A68EB
:106DE00082434A607047000000700040024801681A
:106DF00082151143016070470070004002494A68E3
:106E000002434A6070470000007000400548016876
:106E10000222114301600448016904221143016107
:106E200030BF70470070004000ED00E00A4B1A6868
:106E30009208920002431A6008480369042213432F
:106E40000361012906D040BF20BF20BF01699143E3
:106E50000161704730BFF9E70070004000ED00E0CD
:106E6000F8B504460078544D800672D5524E00277E
:106E7000403EB06BC00004D4B06BA9050843B063BA
:106E800001274E480168C90511D4016882151143D4
:106E90000160FFF731FD009005E0FFF72DFD00993F
:106EA000401A642837D845480068C005F5D53268CF
:106EB0000321090560680A400140914208D081031E
:106EC000890F032904D13168890301D50120F8BD58
:106ED0002A69032109040A4022D0084090421FD0A9
:106EE000207880061CD528692A6988430121C904B5
:106EF0000A432A612A698A432A612861C0050FD59D
:106F0000FFF7FAFC009008E0FFF7F6FC0099411A41
:106F10002B48814201D90320F8BD28698005F3D5AB
:106F200061688803800F032805D132680005824319
:106F300001400A433260286903226168120411404B
:106F400008432861002F04D0B16B01200007814362
:106F5000B1632078C00705D0E868A1688008800088
:106F60000843E8602078800705D5E8680C2188434D
:106F7000E1680843E8602078400706D5E868032107
:106F80008902884321690843E8602078000706D514
:106F9000E86803210903884361690843E8602078B1
:106FA000000606D5E868032189048843A1690843DF
:106FB000E8600020F8BD0000401002400070004072
:106FC00088130000F8B50E4605007DD053480068D0
:106FD000C007C00FB0420AD25048016849084900B2
:106FE000314301600068C007C00FB04271D12878FA
:106FF0004B4C800705D5E068F0218843A968084319
:10700000E0602878C00752D06868022817D00328AB
:1070100018D02168012818D08905002959DAE168BB
:10702000890889000143E160FFF766FC696807464B
:10703000022912D003291CD0012926D033E021686F
:107040008903EAE721688901E7E74907E5E7FFF7F0
:1070500053FCC11B3348814223D8E0680007800FEE
:107060000228F4D123E0FFF747FCC11B2D488142E1
:1070700017D8E0680007800F0328F4D117E0FFF766
:107080003BFCC11B274881420BD8E0680007800FFA
:107090000128F4D10BE0FFF72FFCC11B21488142EE
:1070A00001D90320F8BDE0680007800FF3D11B4829
:1070B0000168C907C90FB1420DD9016849084900E3
:1070C00031430160006800E003E0C007C00FB04238
:1070D00001D00120F8BD2878400706D5E0680721D7
:1070E00009028843E9680843E0602878000707D56B
:1070F000E0680721C90288432969C9000843E060A4
:1071000000F036F8E168084A0906090F515CC840EA
:10711000064908600020FFF711FCF8BD002002407E
:107120000010024088130000C2AA00081C010020C1
:10713000044805490068C968044A4905490F515C7B
:10714000C84070471C01002000100240DBAA000864
:10715000044805490068C968044A8904490F515C1C
:10716000C84070471C01002000100240DBAA000844
:1071700010B5184AD1680C20084004280BD0082804
:1071800010D00C2810D050680004410F0120C0031B
:10719000491C884010BD1068C00601D50E4810BDBE
:1071A0000E4810BD0E4810BD88020E4B000F185C33
:1071B0000902D368890F491CDB0301D5084A05E0A1
:1071C0001268D20601D5044A00E0044A5043FDF794
:1071D0008FFF10BD0010024000093D000024F400A4
:1071E00000127A00D2AA0008FEB505007ED0FE4C3F
:1071F000E7680C20E6680740012000040640287874
:10720000C00747D0082F05D00C2F0AD10120000459
:10721000864206D1206880033CD568680028E5D006
:1072200038E0012069680004814203D121680143EC
:10723000216011E0052301221B0492049942216878
:1072400002D111432160F1E78143216021680140AF
:107250000091206890432060686800280DD0FFF7F7
:107260004BFB009005E0FFF747FB0099401A6428AC
:107270007AD820688003F6D50CE0FFF73DFB00903C
:1072800005E0FFF739FB0099401A6428F0D8206820
:107290008003F6D42878800755D50923E868042FA1
:1072A0000DD00C2F01D1002E09D000283BD0216831
:1072B000994301432160FFF71FFB064627E0216841
:1072C000490701D5002891D061681F22120291431D
:1072D0002A691202114361602168994301432160C8
:1072E000FFF746FFE16809060A0F00E079E1BF49B0
:1072F000895CC840BE4908600020FFF71FFB0028DA
:1073000072D120E0FFF7F8FA801B0228B0D820687D
:107310004007F7D560681F210902884329690902DF
:10732000084360600FE02068400840002060FFF7DD
:10733000E3FA064604E0FFF7DFFA801B022897D83D
:1073400020684007F7D42878C0065FD5002F0CD0FE
:10735000A869002849D02068FF2101310843206036
:10736000FFF7CAFA06462DE0C0E02068800502D586
:10737000A8690028A7D06068072149038843296AC3
:10738000084360606068297F0002000A090608431C
:107390006060286A410B0120C003491C8840E168F5
:1073A00009060A0F9149895CC8409149086000208C
:1073B000FFF7C4FA002817D128E0FFF79DFA801BD9
:1073C0000228A3D820688005F7D560680721490303
:1073D0008843296A084360606068297F0002000AC8
:1073E00009060843606011E0E1E02168FF200130F8
:1073F00081432160FFF780FA064604E0FFF77CFA3C
:10740000801B022872D820688005F7D42878794E2E
:10741000000724D568690028306910D0012108438D
:107420003061FFF769FA009005E0FFF765FA00990F
:10743000401A02285AD830698007F6D50FE0400874
:1074400040003061FFF758FA009005E0FFF754FA6A
:107450000099401A022849D830698007F6D4287864
:10746000400765D500200290A06BC00006D4A06B39
:10747000012109070843A063012002905E480168CA
:10748000C90511D40168821511430160FFF734FA70
:10749000009005E0FFF730FA0099401A642825D8DB
:1074A00055480068C005F5D5FF20AA680130824222
:1074B00003D131690143316111E001218902002AC0
:1074C00007D005231B029A4203D132690A43326175
:1074D000EFE7326982433261306988433061A868DE
:1074E00000280FD0FFF708FA009007E05EE0FFF7F2
:1074F00003FA0099411A4148814257D83069800502
:10750000F5D50DE0FFF7F8F9009006E0FFF7F4F984
:107510000099411A3948814248D830698005F5D42C
:107520000298002804D0A06B012109078843A063BA
:10753000686A002864D00C2F3ED001263606022847
:10754000206805D0B0432060FFF7D6F905462FE04C
:10755000B0432060FFF7D0F9074604E0FFF7CCF90D
:10756000C01B022822D820688001F7D4E96AA86AE3
:10757000E2680843296BFD231B049A431143084327
:10758000E060206830432060FFF7B6F9054604E06C
:10759000FFF7B2F9401B022808D820688001F7D510
:1075A0002EE0FFF7A9F9401B022801D90320FEBDF8
:1075B00020688001F5D423E00128F8D0E06801219B
:1075C0000904AA6A014091420BD10F218904EA6A99
:1075D0000140914205D1032189050840296B884269
:1075E0000ED00120FEBD000000100240C2AA00081B
:1075F0001C01002040100240007000408813000071
:107600000020EFE770B5040007D00026254640357E
:10761000A662687C002802D005E0012070BD2E74AF
:10762000204600F02FF8022068742068016840228C
:1076300091430160A168606822690843E1681143D1
:107640000843616901220843A169520211400843BD
:10765000E1690843216A0843A16A08432168086078
:10766000A0690421000C0840616A08432168486051
:107670002068C16992009143C16166650120687408
:10768000002070BD10B586B0044614216846FDF791
:107690008EFD10492068884219D10F48416B821431
:1076A00011434163C16A01221143C162C06A0021D2
:1076B00010400590E02000900220019003200390EC
:1076C00002910491052069460007FFF749F806B0CA
:1076D00010BD00000030014000100240094910B503
:1076E000401E884201D9012010BD074C6061032172
:1076F000081F00F0FFFD0020A0610720206100208E
:1077000010BD0000FFFFFF0000E000E07047704781
:10771000F8B502680446D0691168936805072D0F13
:107720005BD0DD07ED0FFF2621360E402E4367D0DC
:10773000C60706D0CE0504D501261662E26F324395
:10774000E267870702220426002F06DADF0704D04B
:1077500027683A62E76F3743E767470706D5DB07D5
:1077600004D023681E62E36F1343E367020709D561
:1077700020220A402A4305D0236808221A62E36FB8
:107780001343E367E26F002A2FD0800606D58806F0
:1077900004D5216E002901D020468847E06F21687A
:1077A0008968490601D4000724D5204601F03AFF34
:1077B00020688168490619D581684022914381601B
:1077C000E06E002812D020498163E06EFEF72EFEA5
:1077D00000280AD0E06E816B06E0850610D58D0684
:1077E0000ED5216E1CE020468847F8BD2046FFF7E5
:1077F0008EFFF8BD2046FFF78AFF0020E067F8BD46
:10780000C50208D55B0206D501200005106220469E
:10781000FFF77CFFF8BD030605D50B0603D5616EA7
:107820000029E0D1F8BD4006FCD54806FAD513681A
:10783000204640218B43136020216167002161664F
:1078400000F069F9F8BD00008195000810B504004A
:1078500003D0606F002802D007E0012010BD002196
:1078600070200155204600F027F82420606720682A
:107870000168490849000160204601F01DFF012808
:10788000ECD0606A002802D0204601F05BFD206841
:1078900041680922D20291434160206881682A220E
:1078A00091438160206801680122114301602046F4
:1078B00001F0AEFD10BD0000F0B587B00646142102
:1078C0006846FDF774FC2C493068884251D12B483A
:1078D000416B0122920311434163C16A01221143AA
:1078E000C162C06A0025104005900320400200904C
:1078F0000220032701A9A1C10420049005206946A4
:107900000007FEF72DFF1F4C1D48A560E56081C4F0
:107910008027E560A7602020256160610002A061EA
:107920001848083CFEF7FCFD002801D0FEF73EF9A0
:10793000F466A662144C12482146143820600320D5
:10794000606010200831A1C16561A561E561204634
:107950002562FEF7E5FD002801D0FEF727F9B466A1
:10796000002201211B20A662FFF734FA1B20FFF73B
:1079700027FA07B0F0BD00000038014000100240B7
:1079800030000240F015002038160020F8B50446FB
:10799000806F20284DD100290BD0002A09D0012367
:1079A000A0681B03984206D12069002803D1C807AC
:1079B00001D00120F8BD25466035287C012838D04B
:1079C000012028745820616502530026E6672220B2
:1079D000A067E06E002819D01749C162E16E174810
:1079E0000863E16E16484863E06E13468663676D70
:1079F00021683A462431E06EFEF7DAFD002805D012
:107A00001020E0672E7420206067D2E72E74206873
:107A10000168FF2201321143016020688168012260
:107A200011438160206881684022114381600020F9
:107A3000F8BD0220F8BD0000DD9500081B96000887
:107A40009595000870477047FFB50446406F83B0B6
:107A500017460D4620285CD1002D0AD0002F08D0F3
:107A6000A168C001814207D12069002804D1E8073C
:107A700002D0012007B0F0BD204660300290007CAB
:107A8000012846D00298012101740020E0672120DE
:107A90006067FEF731FF26464036019037827782D5
:107AA0000120A1680003814202D12069002802D090
:107AB0002F46002511E000270FE0002280212046FC
:107AC00001F00EFF002815D1002F15D0216838785D
:107AD00088627F1C708A401E7082708A019B002819
:107AE00006980090E9D100224021204601F0F8FEDE
:107AF000002808D00320BDE728882168C005C00DF4
:107B00008862AD1CE6E720206067029900200874B7
:107B1000B0E70220AEE7704701490248C160FDE7C7
:107B20000400FA0500ED00E010B50524240700224A
:107B300004212046FEF7D9FE002208212046FEF748
:107B4000D4FE0A2002F0CBF9012204212046FEF7E0
:107B5000CCFE0A2002F0C3F9002204212046FEF7E1
:107B6000C4FE10BD10B505242407002204212046C0
:107B7000FEF7BBFE012208212046FEF7B6FE0A20D2
:107B800002F0ADF9012204212046FEF7AEFE0A20E4
:107B900002F0A5F9002204212046FEF7A6FE10BD42
:107BA000F8B500240526074625463607002204219D
:107BB0003046FEF79AFE0A2002F091F901220421D4
:107BC0003046FEF792FE6006040E08213046FEF7AE
:107BD00083FE002801D0641CE4B2052002F07FF986
:107BE0006D1CEDB2082DE1D3002F03D0FFF79CFFF1
:107BF0002046F8BDFFF7B6FFFAE770B50526054643
:107C00003607002204213046FEF76FFE0024E80903
:107C100001D0012200E0002208213046FEF765FE77
:107C20006806050E0A2002F05AF9012204213046A6
:107C3000FEF75BFE0A2002F052F9002204213046D2
:107C4000FEF753FE0A2002F04AF9641CE4B2082C45
:107C5000DDD370BD10B5052424070122082120467C
:107C6000FEF743FE012204212046FEF73EFE0022DD
:107C700008212046FEF739FE0A2002F030F90022E2
:107C800004212046FEF731FE10BD10B5052424075F
:107C9000002204212046FEF728FE0022082120466B
:107CA000FEF723FE0A2002F01AF9012204212046E1
:107CB000FEF71BFE012208212046FEF716FE0A20D1
:107CC00002F00DF910BD70B505252D070024012225
:107CD00008212846FEF709FE062002F000F90122DD
:107CE00004212846FEF701FE062002F0F8F807E01E
:107CF000641CE4B2FA2C03D9FFF7C7FF012070BD62
:107D000008212846FEF7E8FD0028F1D100220421D1
:107D10002846FEF7EAFD002070BD0000F8B501F02E
:107D2000A7FB01F0E1FB46480068C069FEF72EF8AA
:107D30004449454E898F002914D044490A780121CD
:107D40008902002A0AD0012A04D0022A04D0032A78
:107D500008D103E0212801D2002200E001223046B0
:107D6000FEF7C3FD0121C9023046FEF7B5FD01272C
:107D7000FF03374D0024002825D036480460E879F9
:107D8000002803D10120E87101F0EEFD2878632876
:107D900006D9002208213046FEF7A7FD012205E0A2
:107DA000012208213046FEF7A0FD002205203946B9
:107DB0000007FEF79AFD234D274E4035A88C274F2C
:107DC000012803D01CE0EC710022EAE72448694650
:107DD000088072B680212348FDF700FF002804D0F8
:107DE000022269461F48FDF79DFF62B61EA001F002
:107DF00059FEAC8402F0E6FD642002F069F8FE60F2
:107E0000688C012808D10F486C84048002F0DAFDE8
:107E1000642002F05DF8FE60288C012806D12C84D5
:107E200002F0D0FD642002F053F8FE600548124ACB
:107E30000188914202D1C088002800D1FE60F8BDBF
:107E400070150020500D0020000400506B00002031
:107E5000D4000020100100200400FA0500ED00E02D
:107E6000AAAA0000384A0008BDF8C8EBC9FDBCB694
:107E7000C4A3CABD0D0A0000AA55000008B53721E9
:107E8000202000F06EF80321212000F06AF8402144
:107E9000222000F066F80821232000F062F8AA21D1
:107EA000302000F05EF80A48008FC1B2322000F0A6
:107EB00058F80221332000F054F85F21202000F010
:107EC00050F8684600F006F80A2002F008F808BDED
:107ED000500D002010B501460F2000F021F80028B9
:107EE00000D0012010BD10B50446FFF7B3FE3220CC
:107EF000FFF783FEFFF7E7FEE0B2FFF77EFEFFF736
:107F0000E2FEFFF7A7FE3320FFF777FEFFF7DBFE69
:107F10000020FFF745FE0446FFF7B7FE204610BDE0
:107F200010B50C46FFF7DFFF2070012010BD70B5C3
:107F30000D460446FFF78EFE3220FFF75EFEFFF788
:107F4000C2FEE0B2FFF759FEFFF7BDFE2846FFF77D
:107F500054FEFFF7B8FEFFF798FE0A2001F0BFFFBE
:107F600070BD10B5FFF7E3FF012010BD10B502484A
:107F7000FEF704FE10BD0000E8140020FEB5044624
:107F8000002572B60068394A831804D13849CD6893
:107F9000032189040D4081680191C1680091416904
:107FA0008669002B08D132484038836AC7043B43B6
:107FB0008362836ABB4383620846304348D02B48C0
:107FC0002368C34205D12A48C3680322920493431D
:107FD000C360002917D02068026901231A43026197
:107FE00020684161FEF788FC0746FEF785FC2168A2
:107FF000C01B0968090703D47D21C9008842F4D950
:10800000216808204860002E17D0206801690122ED
:108010001143016120688661FEF76EFC7D270646EC
:10802000FF00FEF769FC2168801B0968C90601D4BE
:10803000B842F6D92168102048600C482168C14236
:1080400006D10B48C1680322920491432943C160C1
:108050002068016949084900016121680198886028
:1080600021680098C86062B6FEBD00000084FFBFB2
:10807000401002401CB5002116480091144A01919D
:108080000260C1631205426081600722826301229F
:1080900002610246C16020321170FF235170C23369
:1080A0004362816211730163816104224163426111
:1080B000C161FEF721F808480090801301906946DD
:1080C0000448FDF7C9FF00210248FDF76FFF1CBD02
:1080D000002401408C1400200200000408B5084868
:1080E000016B012211430163006B012110400090DC
:1080F00000220A20FEF76EFE0A20FEF761FE08BD90
:1081000000100240F0B587B014216846FDF74FF823
:108110004C48C26A04210A43C262C26A0A400592FC
:10812000C16A80273943C162C16A39400591C16A79
:1081300001252943C162C16A29400591C16A02260D
:108140003143C162C06A2A463040059005201C2197
:108150000007FEF7CAFB01223B493C48FEF7C5FB7E
:1081600000223B493948FEF7C0FB9121052000223F
:1081700009020007FEF7B9FB3648019000240520EC
:108180006946009502940007FEF7EAFA0320019081
:1081900005206946009602940007FEF7E1FA0C20DC
:1081A000009011200190032003900520029469465D
:1081B0000007FEF7D5FA10200090052069460396C7
:1081C000019502940007FEF7CBFA1120019002946A
:1081D0006946009503941D48FEF7C2FA1E480190B7
:1081E0006946009602951948FEF7BAFA1B480090B6
:1081F00002946946019503941448FEF7B1FAE80227
:108200006A4651C269461148FEF7AAFA9120000257
:108210000090052002946946019503940007FEF73B
:108220009FFA69460948009702950194FEF798FA6B
:10823000002201210520FEF7CDFD0520FEF7C0FD3F
:1082400007B0F0BD0010024001060000000400501D
:108250000830000000001110000021100836000056
:1082600010B50F4C0D482060FF20053060600020E5
:10827000A060E06020616061E0610121206249024C
:108280006062A161A0620720E0622046FFF7BAF9B0
:108290002068016840221143016010BD0030014098
:1082A0001815002000B585B014216846FCF77FFF43
:1082B0000E480D490160E1214902416000218160C1
:1082C000C160016181610C22C161426101623021A2
:1082D00041620121090381634900C163FFF7B6FAD6
:1082E00001F03CFB05B000BD0038014070150020D6
:1082F000704700008307FF22DB0E9A408907090EB2
:10830000994000280BDA0007000F08388308084856
:108310009B001818C36993430B43C36170478308DC
:1083200004489B001B181868904308431860704766
:1083300000ED00E000E400E0BFF34F8F0449034884
:10834000C860BFF34F8F00BFFDE700000400FA05CF
:1083500000ED00E0FEB50A2002F0AAF87D20C00082
:1083600002F0C0F8FC4C0025A570E07B0C2801D37E
:108370000B20E0730122052051020007FEF7B5FA39
:108380000026F648E670F64D00782871F549A07988
:10839000097840000843617D89000843E871E06A7C
:1083A000E870401CE06260792946A8744200B4314C
:1083B0000846A138FCF7E2FE06206872EA48E64962
:1083C0000078A872207F2873284613388A7F0275A8
:1083D000C97F41756079002240002946153002F0BE
:1083E00051F9607900214000153002F05DF902205A
:1083F00002F0AEF8EE716674E672012060732673C7
:10840000DA48FEF79BFC60840546E6706079FDF76C
:1084100035F9D74AD74BFDF72BF801F0F5FC0123CE
:1084200000229B07FCF772FFFDF76EF90006C10CF6
:10843000481980B20121C903A084884201D3401A9F
:10844000A084CD48A0632079401C2071C748FEF766
:1084500075FC2084C2480C300646423640300190FC
:1084600074E1C248FEF76AFC2084C44FC44D0AE0A0
:10847000BE48FEF763FC80B22084A18C884202D300
:108480004919884206D300210F2001F091FF38429C
:108490002063EDD0206B2546411C20D040047DD5C3
:1084A0008122D20100210F2002F0C1F87D20C000FE
:1084B00002F018F8002001F0CAFF0021102001F09E
:1084C00077FF4106A648490E00225030A96401F00A
:1084D000A5FFA3485030417A0729C1D101E0FFF739
:1084E0002BFF0222A749401DFCF76CFE0028B7D1E4
:1084F00002F02BF96965286502F014F9E965A865B1
:10850000E8786946401CE87095484D3002790A7059
:10851000407948700888E98B884275D19A4D308A35
:10852000288001988C49808A48839048FEF706FC91
:10853000208401F04FFEFF23A16D5B04E06D00225B
:10854000C918504100060F0A074378084000010E81
:108550000002616620668248636D0A30226D02F077
:10856000C9F86079E36D81007D48A26D0818163066
:1085700002F0C0F87A48636E1230226E02F0BAF848
:1085800077480821417260790022800074491C30CC
:1085900002F078F860798000002100E0C9E01C302A
:1085A00002F082F8384601F07CFF012001F0D0FF94
:1085B000607202217548FEF78FF9002825D000204F
:1085C000684908706448B1898186F289C286606B07
:1085D000A06363485030C37C1E07360F032E00D0C3
:1085E000E6741B0923750026267101265A4FE67290
:1085F00039877A87002B16D002226249401DFCF78A
:10860000E1FD002803D00EE075E00120D8E75448D2
:108610006674C671A06C52491638C2B2A274663133
:108620005B48FCF7ABFD2673608B5A49FF30C330C3
:1086300080B2608388420CD9494240186083288800
:108640007D21401C80B2C9002880884201D30020CF
:1086500028802D887D20C000618B68434018E0632E
:1086600000904D48302107784C48277400884843D3
:10867000FCF7E9FF019028460A214843FCF7E3FF95
:108680000199FCF705FE7F21C905FCF7A8FDFDF760
:1086900003F880B240497F1E0880B84200D126739B
:1086A000E5841620205EFCF7D5FF07460191208C5B
:1086B000FCF7E4FF3A4A3B4BFCF7DAFE05460E4670
:1086C0000098FCF7C7FF2A463346FCF7C3FE3A463C
:1086D000019BFCF71BFEFCF7F3FF2064A08B00F06E
:1086E0001BFD607A002863D100210F2001F060FE9D
:1086F0000006F9D55CE0FDF731FB254903220C3972
:108700000A541549B2898A86F289CA8620498000AE
:10871000CC3942180199098B11801D496A6B9C392B
:108720000A500F49EB6D40181630AA6D01F0E2FFB8
:108730000CE03A4600210F2001F079FF6879E978D2
:10874000401C814202D0002001F081FE208CA18CCF
:10875000884229D285E6000058000020D40000207D
:10876000C41100200C010020E4000020E8140020C7
:10877000B81E85EB51B8CE3FA086010000D027245B
:10878000983A0000F4000020080100200004005086
:1087900074130020E7030000EA000020EE00002030
:1087A000F853E3A59B843E40614A89188842D1D89A
:1087B00001F010FD5F4A00210F2001F038FF5E48F4
:1087C00000250078002802D1A08B00F0A5FC002035
:1087D000E073627921E0584E315C00291BD0E37BC5
:1087E000AE005B1CE373544BB446303B9951524E80
:1087F0004300F03EF65A6F004F4B6D1CD83BDE53E2
:10880000860048334C4F9B596646603FBB514A4BEC
:10881000491EEDB21954401CC0B29042DBD3E0783F
:10882000032801D2E07BE07344490022C87B8873AF
:10883000401E32E000212CE03F4C8B00603C1E19B2
:10884000B446E5587668B54221DD01953A4D4C00B5
:10885000D83D2D5B9700AE46374D303DED59009524
:10886000354D603DEE50783D334E67197D88D83EDA
:1088700035533446A8341E192F4D7468303DEC50E2
:108880006346019D5D6075467D80009D7560491C55
:10889000C9B28142D0DB521CD2B28242CADB264826
:1088A000603802682548816B32398A4207DA2249EA
:1088B00030390968002902D0C179491C00E0002143
:1088C000C1711F49C37909884A009A4205D21A4AE0
:1088D000D83A1288C283022202700A2251430279D6
:1088E000914201D200210170407C002806D012493B
:1088F0000C310B7848788A78022B0DD00D4A002174
:1089000080320F2001F093FE012105200022490250
:108910000007FDF7EAFFFEBD0A4BC91C1818FCF75B
:108920002DFC02F04FF8642001F0D2FAD7E50000E8
:10893000983A000000D02724681300205800002037
:10894000E4000020500D002070470000F0B58DB00D
:10895000B54801900020C0430A9000260A2001F08B
:10896000A7FD7D20C00001F0BDFD0020AF4C0546F5
:10897000A070AF4FAF480B90AE480022C23885734D
:108980000146142001F07EFE0021142001F08CFE2F
:10899000022001F0DDFD00210F2001F009FD384229
:1089A0002063F8D0206B411C18D040047ED5812272
:1089B000D20100210F2001F03AFE0021102001F029
:1089C000F7FC41069B48490E0022801C01F026FD61
:1089D0009848801C417A022902D008E1FFF7ACFCDC
:1089E000944802229449C01DFCF7ECFB0028F4D106
:1089F00001F0ABFE6165206501F094FEE165A065C4
:108A0000002E23D10B998D48098A01808948874916
:108A1000801E808A488301268948FEF78FF92084CA
:108A2000608B8849FF30C33080B2608388420DD9A3
:108A300049424018814960830888824A401C80B2BC
:108A40000B320880904201D3002008800B986946C1
:108A500082890A80C089488076490422C91C084658
:108A6000A238FCF78BFBFF22A16D5204E06D0023BE
:108A7000891858410006090A01430846029101F08D
:108A800010FD029948084000010E00026166206650
:108A90006848636D9638226D01F02CFE6548E36DE1
:108AA0009238A26D01F026FE624800E0A1E08E3807
:108AB000636E226E01F01EFE5E490022A0393C204A
:108AC00001F0E0FD00213C2001F0EEFD012001F06D
:108AD0003FFD6072A0780121401CA0700520C903F1
:108AE0000007FDF74FF955487D220188D20008465E
:108AF00050430291628B0A398018E0630C9052480F
:108B000000782074049008B22085002803DA7D21C3
:108B1000C900401820854D48302100884843FCF7A3
:108B200092FD05902820205EFCF782FD0599FCF758
:108B3000AFFB7F21C905FCF752FBFCF7ADFD4249B5
:108B400080B208800499491E884201D10120207317
:108B50000298E0841620205EFCF77CFD05910690CB
:108B6000208CFCF78BFD3A4A3A4BFCF781FC0791CD
:108B700004900C98FCF76EFD079B049AFCF76AFCC6
:108B8000059B069AFCF7C2FBFCF79AFD2064A08BBC
:108B900000F0C2FA00990198814210DA00290ED043
:108BA00024490422C91C0AA8FCF7E8FA0220207014
:108BB00029480A2100784843A07200980190607A01
:108BC000002805D100210F2001F0F2FB0006F9D5A5
:108BD000802200210F2001F02AFD00206D1CEDB243
:108BE0006070032D00D2C7E6002E08D017E00120E8
:108BF000F4E71A4A00210F2001F019FDF7E7A18BD5
:108C00001748002902D00288914201D90188A18326
:108C100088B21449401E09884843134908800A98BD
:108C2000E0830DB0F0BD00003F420F00580000206F
:108C300000D0272412120020F40000200801002098
:108C4000E8140020E7030000EA000020EE00002006
:108C5000F853E3A59B843E40E400002000902724C5
:108C6000E0000020DE000020DC000020F8B53B49D9
:108C70003948086001F046FE2120394C000160802F
:108C8000204640300079374D0006000E687003D052
:108C9000E08800280AD00BE07D20C000E0800120A1
:108CA000E0870A2060870020A08701E06420E08040
:108CB000208F0A2801D902202087E08E3C2801D984
:108CC0003C20E086284980B20870E08F6871A08F50
:108CD000A871A07AE870A68805212E626981E788CC
:108CE0003846FCF705FAA88101463046FCF700FA41
:108CF0008800081886B27D20C0002E817043FCF7E2
:108D0000BDFC1A4A1A4BFCF71BFCFCF7FDFCE88182
:108D10007D206E823946C000FCF7EAF928820146C0
:108D2000C820FCF7E5F968830120E882FDF72EF8FA
:108D3000A882EA890F491048FEF704F80FA0296AB3
:108D400000F0B0FEE18811A000F0ACFE218914A073
:108D500000F0A8FEF8BD0000959900085000002022
:108D6000500D0020D400002000000020F853E3A59F
:108D70009B843E40FF7F0000E8140020B1EAC7A9B1
:108D800049443A202564202E0D0A0000CDA8D1B612
:108D9000BCE4B8F43A202564206D732E0D0A00005F
:108DA000B5A5B4CECDA8D1B6BBF9D5BECAFDC1BF5D
:108DB0003A202564B8F62E0D0A000000F0B5924D59
:108DC00085B001202880914FC820914C3880207AAE
:108DD000401C2072C00706D0A08B411EA183022830
:108DE00001D2C820A083A08B00F096F90A2001F0E0
:108DF0005FFB7D20C00001F075FB02218548FDF777
:108E00006BFD002838D00020834980000978844E0B
:108E100049000843814909780843B07210207072F4
:108E20008048C1887D20C000FCF762F970737E48DD
:108E30007C490078B07330460B308A780270C9786C
:108E40004170411C77482030027ECA70407E087114
:108E500074482230027E4A71407E887100220C39AB
:108E6000152001F00FFC0021152001F01DFC02204F
:108E700001F06EFB6D4E03E00120C5E7FEF74EFFEB
:108E800000210F2001F094FA30422063F6D0206BCD
:108E9000411C7DD040047CD58122D20100210F20CD
:108EA00001F0C5FB0021102001F082FA41065C4868
:108EB000490E00225030A16401F0B0FA584E5036ED
:108EC000707A112865D102225949701DFCF77AF990
:108ED00000285ED1F01E027969460A704079487018
:108EE000B17A2980C820FCF703F93880307BA08351
:108EF000504DB01E008A28804549301F808A488323
:108F00004D48FDF71BFF80B220840390608B4B49D6
:108F1000FF30C33080B2608388420CD94942401888
:108F2000608328884549401C80B20B3128808842E4
:108F300001D3002028802D887D20C000618B6843EC
:108F40004018E06302903E48067828460A3800B28E
:108F500026742085002803DA7D21C9004018208569
:108F6000388830214843FCF76EFB07462820205EF6
:108F7000FCF75EFB3946FCF78BF97F21C905FCF74E
:108F80002EF9FCF789FB2E4980B20880761E01E09D
:108F900037E034E0B04201D101202073E58416208F
:108FA000205EFCF757FB074601910398FCF766FB30
:108FB000244A254BFCF75CFA05460E460298FCF75E
:108FC00049FB2A463346FCF745FA3A46019BFCF733
:108FD0009DF9FCF775FB206468460088E083104823
:108FE0000F495030807C6071420063310846513037
:108FF000FCF7C4F8A08BFF2801D00320207005B037
:10900000F0BDFFF799F90000E4000020EE00002019
:109010005800002000040050D9000020DA00002091
:10902000C4110020500D00200000002000D0272493
:10903000F400002008010020E8140020E7030000ED
:10904000EA000020F853E3A59B843E4070B586B04B
:1090500014216846FCF7ABF801250F4EED03002202
:1090600029463046FDF741FC01200024019002947E
:109070006946009503943046FDF772FB032001908A
:1090800002946946009503943046FDF769FB02207F
:1090900000F01EFF06B070BD0004005070470000D5
:1090A000F8B5044600206A461080194D55222A70F2
:1090B000AA226A700322AA70661DEE702A71697175
:1090C000144A49008918AC712246E81DFCF756F88D
:1090D000002007E029186A468978128889186A46AC
:1090E0001180401CB042F5DB611DA81CFCF7A2FCFE
:1090F00001466846018029190078C87168464078A1
:10910000087221460931024800F0A4FAF8BD0000B7
:1091100028140020500D002010B51B4CE18A228A33
:10912000914201D3891AE18289B2628B0B46534383
:109130001B182383132902D14A4310182083208B44
:10914000302148436421643048431049E062096893
:10915000401A0F494018A062FCF77CFA0D4A0E4BEA
:10916000FCF7EEF9FCF7ACFA0C496062884202DDCC
:109170004A4280186062002801DA4018606208499B
:109180000968486110BD0000D4000020980000204C
:10919000F0D8FFFFF853E3A59B843E40FF7F00001B
:1091A000E8140020034A1168382389B29943014327
:1091B000116070470030014010B5FDF7A3FB10BDF2
:1091C00010B59AB034216846FBF7F1FF14210DA8C1
:1091D000FBF7EDFF1C2112A8FBF7E9FF1B48016814
:1091E0000324E402A143C21489180160FDF7FEFDC7
:1091F00017480169A143016106200090FF2001305A
:109200000290012003901020049002200990400455
:109210000B90000100240C900A946846FDF7E4FFCF
:109220000F200D9003200E900F94109401211194A3
:109230000DA8FDF7C7FE812012900320800418902E
:10924000149412A8FDF70CFE1AB010BD0070004077
:109250004010024010480168821511430160C16846
:109260000E4A1140C16001680D4A114001608168D9
:10927000490849008160016801229204914301601C
:10928000C168FD2212049143C160002101610649B9
:109290000448886070470000001002400C40FF88BE
:1092A000F6FFF6FE0050000800ED00E070B501F09A
:1092B00093F8224C224DE06402E001F08DF8E06466
:1092C000A842FAD1207801260525F6032D070028AB
:1092D00006D001280CD0022817D003282BD128E073
:1092E000012231462846FDF700FBFFF767FD06E047
:1092F000012231462846FDF7F8FAFFF727FB002246
:1093000031462846FDF7F1FA15E0A07A0122401E09
:10931000A07231462846FDF7E8FAFCF753FD00221B
:1093200031462846FDF7E1FAA07A002803D12070E3
:1093300001E0FFF70FF800F035FF70BD5800002086
:109340003001CADE10B5818CC90707D001684A68B0
:1093500001235B049A43836A1A434A60818C89071C
:1093600007D501684A6801231B049A43C36A1A435C
:109370004A60818C490707D501684A6801239B042C
:109380009A43036B1A434A60818C090707D5016829
:109390004A680123DB039A43436B1A434A60818C7A
:1093A000C90607D50268916801231B039943836BA3
:1093B00019439160818C890607D501688A68012369
:1093C0005B039A43C36B1A438A60818C490612D5AA
:1093D00003685A6801210905046C8A4322435A60D4
:1093E000026C8A4207D10268516803235B059943E6
:1093F000436C19435160818C090607D501684A689E
:109400000123DB04806C9A4302434A6010BD0000D4
:10941000F8B500260446C667FDF76EFA05462068D3
:109420000068124F000709D501212B46002249058B
:109430002046009700F054FA00280DD120680068FB
:1094400040070BD501212B460022890520460097B5
:1094500000F046FA002801D00320F8BD2020606704
:10946000A067603426740020F8BD0000FFFFFF01F4
:10947000F8B5184CC826E078002829D16079002872
:1094800026D101206071144D686B002700281ED082
:10949000686BC821081A15E01048E168405C6169F2
:1094A00088470F480A21008848430E490880E06831
:1094B000401CE060E068C82800DBE760696BC820FA
:1094C000401A761EE168814201D0002EE4DC67710B
:1094D000F8BD00003C00002000000240880C002085
:1094E000E4000020F000002070B5224CE078002855
:1094F0003FD1207900283CD1012020711E4EF16916
:1095000000250906002933DA2156625791420AD113
:10951000F06940062CD5A079002829D0A5712089B2
:10952000401C208124E0A179002903D1A0710A20E8
:1095300000F0D5FC00202056CC2148430F494218AA
:10954000206912181279B262401C00222061A256D2
:10955000CC235A43895881420ADC25612078401C7B
:10956000207020780E2800D12570A078401CA070B3
:10957000257170BD3C0000200038014060010020D2
:1095800010B5806A0022014640314A834A82FEF7C4
:10959000BEF810BD70B5846A606FA56F21688968D8
:1095A00000260906002906DA212804D15220065394
:1095B000204600F047F820688068400606D5222D36
:1095C00004D15A200653204600F02CF8E06F1021F9
:1095D0000843E0672046FEF79AF870BD10B50146D3
:1095E0000968806A0968890614D400225A210A523F
:1095F00001680A68FF2301339A430A6001688A6898
:10960000520852008A6001688A6840239A438A603F
:1096100020218167FEF716FA10BD10B5806AFEF7AB
:1096200012FA10BD01680A68FF2321339A430A60C9
:1096300001688A68520852008A60202181670021EF
:109640000166704701680A68C0239A430A602021B6
:109650004167704770B5164CE278002A0CD1227928
:10966000002A09D10122E2700025C82903DC022268
:10967000A256002A01DCE57070BD0123E356CC221E
:1096800053430C4AD1500123E356CC2673439B1815
:109690000A460146181DFBF771FD6078401C60709A
:1096A00060780E2800D16570A078401EA070E2E7B7
:1096B0003C00002060010020F8B504462669A2683D
:1096C000E76932436669102000253E432368324330
:1096D00078491E68784F3E4016431E6023685A68DA
:1096E00003263603B243E66832435A602368A26910
:1096F0008B4201D0266A32439E680B273F02BE434D
:1097000016439E606D4E23686D4AB3420CD1D268F9
:109710009207920F06D0012A38D0022A34D0032AA9
:1097200020D11EE001201DE0664EB3420AD1D2686E
:109730000C26324026D0042A28D0082A24D00C2A0D
:1097400010D10EE08B420DD1D66803229202164052
:1097500018D001229202B61A18D0B61A14D0964226
:1097600000D10820564A0126403A574FF6038B4253
:1097700036D100280CD002280DD0042812D0082899
:109780001FD11CE00020EDE70220EBE70420E9E711
:10979000FDF7CEFC08E01068C00601D5384605E0AC
:1097A0004A4803E0FDF7E4FC002873D062685100EA
:1097B0005118814205D81103814202D303E030469B
:1097C000F4E7012566E0010E060250080023301878
:1097D0005941FBF7A3FC03210902411A3C4A55E019
:1097E000E169B14232D1030000F083F909070A0DA3
:1097F00006250606062B0600E3E7FDF799FC1CE0AC
:10980000FDF7A6FC19E010686168C00602D548089B
:10981000304A01E0304A48088018FBF769FC80B202
:1098200001462E4A10399142CBD8511C0140000705
:10983000400F08432CE0FDF79BFC616840004A089C
:10984000EAE76168012248081204E5E7030000F036
:1098500050F909070A0D06260606062C0600B0E791
:10986000FDF766FC1DE0FDF773FC1AE01068616807
:10987000C00602D54808C01902E014484A0810186A
:10988000FBF736FC80B20146144A1039914298D851
:109890002168C8600020206660662846F8BDFDF794
:1098A00067FC61684A088018EAE76168480880191F
:1098B000E6E7000000480040F369FFEF0038014090
:1098C000401002400044004000093D000024F40024
:1098D000FFFC0F0000127A000048E801EFFF0000D3
:1098E000FFB581B017460E4604460A9D09E0681C84
:1098F00007D0FDF701F80499401AA8420CD8002DB2
:109900000AD02068C1693046884318D00020B84288
:10991000EDD0002005B0F0BD20680168FF22A13223
:1099200091430160206881684908490081602020D6
:109930006067A0670020603420740320EAE70120FC
:10994000E5E7000010B504491020096808620248E4
:10995000FDF7DEFE10BD00007015002001490D204E
:10996000887070473C00002010B507480A22018A21
:1099700051438183FEF7B2FBFEF794FCC8220349F2
:109980000348FEF703F810BDD4000020880C002027
:1099900070150020F8B53E4C002321783D4A1D4645
:1099A000082910D0072947D0062950D0052952D0C0
:1099B000042953D0032954D0002956D0012958D066
:1099C00002295AD05BE0A17800264A1F04E0314FFB
:1099D000BF5DFB189BB2761C9642F8DB667927794F
:1099E0009A195118E3786278C9188918C91940186A
:1099F000C0430006000E1AD1012E14D0022E16D13B
:109A000025482449C018FBF7B9FB00F0DBFF6420B0
:109A100000F05EFABFF34F8F21492048C860BFF3C2
:109A20004F8F00BFFDE759081046FFF739FB25703F
:109A3000E570A570A571F8BDA1795054491CC8B254
:109A4000A071A178491F8842F5D1082001E060701B
:109A500007202070F8BDE0700620FAE7607105204D
:109A6000F7E7A070E5700420F3E7552807D101203F
:109A7000EFE7AA2803D10220EBE7032803D02570E3
:109A8000E570A570F8BD032020702071F8BD0000BE
:109A9000CB000020C4130020500D00200400FA0564
:109AA00000ED00E00FB410B503A9044B044A02987E
:109AB00000F002F910BC08BC04B018470DA700085C
:109AC000200100202021020C01D010211046020AA2
:109AD00001D010460839020901D01046091F82083A
:109AE00001D01046891E420801D0881E7047081A0E
:109AF000704730B47446641E2578641CAB4200D2B3
:109B00001D46635D5B00E31830BC184702E008C8DF
:109B1000121F08C1002AFAD170477047002001E0E7
:109B200001C1121F002AFBD1704708B50021684609
:109B300001706B46012202212C2000F087FD0221DA
:109B4000684601706B4601222C2000F07FFD08BDA5
:109B500038B504466D20694608706B4601220749F6
:109B60002E2000F073FD0649002C01D0054A00E0CC
:109B7000054A2E2000F050FD38BD00000608000008
:109B800006180000070600000716000038B5044656
:109B90006B4602220021362000F024FCB321230072
:109BA000FFF7A7FF0E0F08153A3A3A3A1C273A3A40
:109BB0002F34483A00216846017040784108490036
:109BC00014E06946087880088000401C04E069467B
:109BD000087880088000801C08701DE068460278C4
:109BE0000A40483202704178802001436846417043
:109BF00012E0684602780A40027040784106490E39
:109C0000F4E7694648780221084303E0694648784A
:109C1000FD210840694648706B460122002136202C
:109C200000F014FD012200AB11463620013300F094
:109C30000DFD38BD69460878CF21084069462030BF
:109C4000CAE708B5032168464170012101706B46DF
:109C500002220021362000F0F9FC0122D203062165
:109C60002D2000F0D9FC012000F032F90120FFF78F
:109C70008DFF08BD08B5020A69464A7008706B4638
:109C8000022204212D2000F0E1FC03206946087027
:109C90006B46012206212D2000F0D8FC00206946E9
:109CA00008706B46012206212D2000F0CFFC0A210E
:109CB0002D2000F07DFB08BDFFB58DB004460025CA
:109CC00006E025280AD0109A0F999047641C6D1C55
:109CD00020780028F5D1284611B0F0BD00270121D9
:109CE000484A009700E00743641C23780846203B5D
:109CF00098401042F7D120782E2817D1042007432E
:109D00006078641C2A280CD10E98641C02C800914B
:109D10000E900BE000990A22514330394018641C20
:109D200000902078014630390929F3D9207800289D
:109D3000D1D0642808D0692806D075281ED0109A82
:109D40000F9990476D1C5BE00A200E99019001C9A4
:109D50000E91002802DA40422D2102E0390504D597
:109D60002B216A461172012103E0F90704D020215A
:109D7000F7E70BAE0B910DE00021FAE70A200E99F0
:109D8000019001C90E91F7E70199FBF7B1F9303164
:109D9000761E31700028F7D103A8801B2030019077
:109DA000780701D5009801E00120009001998842D0
:109DB00001DD401A00E000200027009006E002A824
:109DC000109AC05D0F9990476D1C7F1C0B988742BD
:109DD000F5DB04E0109A30200F9990476D1C009934
:109DE000481E00900029F5DC05E03078109A761CBA
:109DF0000F9990476D1C0199481E01900029F4DCD1
:109E0000641C65E709280100F8B54A002B4B520D88
:109E1000D6182B4A0C460546142E2BDA002E12DAE1
:109E2000284BFBF773FA00221346FBF799FD40D24B
:109E3000002C03DA0124E40700253AE020462843F9
:109E400037D0214C14E0214F0B46F7403B402B43C9
:109E500031D01C4BFBF75AFA00221346FBF780FD6A
:109E600027D2002C03DD01200005F0400419BC437B
:109E700000251EE0332E1EDC33460027143BFF4333
:109E8000DF40384217D00F4BFBF7EAFA00221346A7
:109E9000FBF766FD0DD2002C0ADD142E0CD0342009
:109EA000811B012088404019A84200D2641C05464D
:109EB000BD4321462846F8BD641CF9E701FCFFFFBD
:109EC0009C7500883CE4377E0000F03FFFFF0F00E8
:109ED0007D2110B5C900484300F001F810BD0021F4
:109EE00040E000BF00BF00BF00BF00BF00BF00BF19
:109EF00000BF00BF00BF00BF00BF00BF00BF00BF6A
:109F000000BF00BF00BF00BF00BF00BF00BF00BF59
:109F100000BF00BF00BF00BF00BF00BF00BF00BF49
:109F200000BF00BF00BF00BF00BF00BF00BF00BF39
:109F300000BF00BF00BF00BF00BF00BF00BF00BF29
:109F400000BF00BF00BF00BF00BF00BF00BF00BF19
:109F500000BF00BF00BF00BF00BF00BF00BF00BF09
:109F600000BF491C8142BCD370470000FEB50446C7
:109F70000020019000906079734940000E5A61788A
:109F80002578491E7148CFB20163042D77D0072D83
:109F900075D000210291217801736C49E379012287
:109FA00092058969002B6CD0914381616748217AC1
:109FB0004173217A82698907890B0A4382610021F2
:109FC000042000F034FB324661492E2000F024FBCF
:109FD0003846FFF7BDFD5F4E0522705D81004018D9
:109FE0005D49431807212B2000F030FB5B490298A4
:109FF00001220B180B21282000F028FB705D584926
:10A0000080000A580C21282000F011FBE079554906
:10A0100080004018A1794900425A0221272000F00F
:10A02000FBFA51487E00825B0421272000F0F4FAFD
:10A03000E079002829D0A07804282CD0282069466F
:10A04000087220220621272000F0E6FA02AB012246
:10A050002621272000F0FAFA444938014018E17817
:10A06000890042580821272000F0E1FAA17A601CFB
:10A07000627A0902114313D016E000E001E00121E9
:10A0800088E71143F608816190E7642206212720C2
:10A0900000F0C2FAE0E71020694608720246D1E7F4
:10A0A00033490172090A4172417A007A0A02024375
:10A0B0002021272000F0B0FA2E4F0C2123203A68EF
:10A0C00000F0B5FAF01982880421232000F0A4FAE8
:10A0D000A07900280BD0E0792749012243180021FC
:10A0E000212000F0B3FA03200190012000902A07FC
:10A0F000120F10010243607800218007000B024319
:10A100000198000502430098400402432079C006EC
:10A11000400902436079C00602431F2000F087FA1D
:10A12000A07861780123084302040848DB03026138
:10A13000E179490319430A4302610021082000F034
:10A1400076FA0020FEBD000090AA0008240100203D
:10A150000428000038AA00080C0000202A00002073
:10A1600040AA000860AA00086CAA000870AA0008AB
:10A170004110000058AA00082C00002038B50C46F9
:10A1800007498A8B002102432C2000F045FA6846DB
:10A1900004706B46012206212C2000F057FA38BDCE
:10A1A0002401002010B5FFF7C0FC10BD10B5044617
:10A1B0000421362000F0FCF80121C902002C01D056
:10A1C000084300E0884302460421362000F02FFABD
:10A1D00010BD000038B540206946087000210E20EF
:10A1E00000F0E6F80446002211460E2000F01FFAA7
:10A1F0006B46012200210D2000F028FA074A0021B9
:10A200000F2000F014FA00F0EDF9224600210E2094
:10A2100000F00DFA02480021017338BDF8FF272431
:10A2200044010020FEB50546042069460870514CE3
:10A230000020607521462031206348710873A08397
:10A240006063A06300F0C8F84B4E206002E000F0AD
:10A25000C3F82060B042FAD10020FFF797FC00F06D
:10A26000BBF8464E20603078242801D9243806E017
:10A270000621FAF73DFF0622101A400108430206A4
:10A2800001040A4301020A430243B26070600021E4
:10A290001E2000F0CCF900F09FF820606B460122F0
:10A2A0000021242000F0D2F91E20FFF7E3FC86B243
:10A2B000300AA0730420FFF7DDFC074600F08CF89D
:10A2C00020603806000E0DD002206946087101ABEF
:10A2D000012212212D2000F0B9F9A08B01210903E0
:10A2E0000843A08300F078F820600620FFF7C2FC46
:10A2F00060600720FFF7BEFCA060F006C00E20756E
:10A3000001D110202075C0B200F0DCF9E80707D0B9
:10A31000FFF797FCA08B0121C9020843A0830AE044
:10A320000521362000F02EF8154908400246052187
:10A33000362000F071F90120FFF728FC00210420ED
:10A3400000F036F8A0610021262000F031F8152138
:10A350008903084302460021262000F068F9002204
:10A360002621362000F058F900F036F82060002051
:10A37000FEBD0000240100203001CADE00000020E4
:10A38000FFFD000038B5094C89B280B26B4602224D
:10A3900000F028F8002806D1684640780102684697
:10A3A0000078081884B2204638BD0000FFFF000086
:10A3B00038B50024E44389B280B26B46042200F031
:10A3C00011F8002806D103216846435C2202D41804
:10A3D000491EFAD5204638BD10B500210846FFF7C2
:10A3E000E7FF10BD38B5002909D0402420436C4652
:10A3F0002070C8B27F2906D8607002200AE0694642
:10A400000870012006E0802420436C466070C80973
:10A41000A0700320694600F0AFFA38BD10B51446AD
:10A4200003460A4621461120FFF7DCFF10BD10B598
:10A430000346052200211520FFF7D4FF10BD10B5FB
:10A440000346052200211720FFF7CCFF10BD38B5C9
:10A45000054600206946087000F0C4F8FF24013466
:10A460002246002D01D00322120200210D2000F00F
:10A47000D3F8002D13D06B46012203210F20FFF7E4
:10A48000B1FF68460078000709D5FFF7A3FE224612
:10A4900000210D2000F0C0F80020C04338BD00208E
:10A4A00038BD10B5024601210A2000F0C0F810BDE9
:10A4B00010B5044600211A20FFF77AFF000D220391
:10A4C0000005120B024300211A2000F0B0F810BD65
:10A4D00010B5024602492E2000F09EF810BD000083
:10A4E00004180000F8B505466B460122032104203C
:10A4F000FFF778FF0126114C3607002D0DD02A46B4
:10A5000000210C2000F088F86946087810210843E3
:10A5100069460870A069304307E069460878EF2172
:10A52000084069460870A069B0430B46A06101224B
:10A530000321042000F08AF8F8BD00002401002067
:10A5400010B502460021182000F066F810BD00008A
:10A55000F8B50746002568460570B807204C2E461A
:10A5600000280ADA8020694608706B460122002123
:10A570000D2000F06BF801202073F8076946087879
:10A5800021D006210843694608706B46012200214C
:10A590000D2000F05BF803210F20FFF7F3FE81216F
:10A5A000C900084219D04020694608706B46012254
:10A5B00000210D2000F04AF80020FFF7F7FD0025EC
:10A5C0002673ED4309E002210843694608706B4693
:10A5D000012200210D2000F039F82846F8BD0000C6
:10A5E000440100201CB56B46012203210F20FFF718
:10A5F000F9FE684600784022C1091040C9014000B8
:10A60000814208D0012069460871024601AB03214E
:10A610000D2000F01BF81CBD08B56B461A70120A1D
:10A620005A7089B280B2022200F010F808BD38B525
:10A6300000236C46E254120A5B1C042BFADB89B23D
:10A6400080B22346042200F001F838BD38B58024DA
:10A65000002909D0C02528436D462870C8B27F293B
:10A6600007D86870022009E020436946087001207D
:10A6700004E020436870C809A8700320694600F010
:10A68000B7F938BD10B51446012312189B029A423F
:10A6900002D90020C04310BD0B46821E214609206E
:10A6A000FFF7D4FF002010BD10B5054A89051269D7
:10A6B00001430A4300210820FFF7B9FF002010BD25
:10A6C0002401002038B504466B4601220E212B20C0
:10A6D000FFF788FE68460078E10640094001C90E90
:10A6E0000143684601706B4601220E212B20FFF7C3
:10A6F000ADFF38BD10B5002142541C06120A22439A
:10A700001B0A491C0429F7DB10BD000013B5012307
:10A710001A4669460248FDF797F900981CBD0000EB
:10A72000701500207CB5002425466846FFF77FFEA3
:10A7300004206946220E2D02154322020C5C1443AC
:10A74000401EF7D5204629467CBD7CB50024254611
:10A750006846FFF774FE04206946220E2D02154359
:10A7600022020C5C1443401EF7D5204629467CBDCE
:10A77000FCF7D0F8FEF724FDFDF7C4FC3C493D484A
:10A78000002522C005608561C5613B490562C16045
:10A790000838FCF759FAFDF7A1FCFDF783FDFDF73A
:10A7A0005FFDFDF767FC052601223607D103304621
:10A7B000FCF79BF8FEF75AFAFDF760FBFBF79AF9F6
:10A7C000FBF768F90721B015FFF7D8FC2B4C0A21DD
:10A7D000208A01224843A083170339463046FCF7FC
:10A7E00084F82448C82226498830FDF7CFF8254E42
:10A7F0002079002839D06078002836D0FEF7E0FCB8
:10A800002571FBF75FFB20700F2809D9012239461B
:10A810003046FCF76AF8FEF749FD0022394609E0A8
:10A82000012251033046FCF760F8FEF73FFD00229D
:10A83000012149033046FCF758F8FDF76FFAA08B69
:10A84000002801D0401EA0830F48A18B0078084348
:10A85000CED10121C9023046FCF73EF80028C7D10D
:10A8600001210846FCF7E2FAC2E7FDF757FABFE715
:10A87000007C0040E8140020FFFF0000D40000200E
:10A88000880C0020000400504200002010B586B063
:10A890001748FCF75EF914216846FAF788FC15485A
:10A8A00000900320019000200290052069460007D7
:10A8B000FBF756FF69461048FBF752FF69460F4801
:10A8C000FBF74EFF01210846FCF7B0FAFF240134E4
:10A8D0002046FCF783FA0A490868042210430860FE
:10A8E0002046FCF78BFAFCF791FA06B010BD000089
:10A8F000E8140020FFFF0000000400500008005092
:10A900000070004010B50122920218491848FBF768
:10A910007FF91648174902888A4226D001807D2196
:10A92000C90081804910C1800A21018100211E22B5
:10A930004181D24382810122C2810184018241820C
:10A940008182C182018381831E23C3860223038700
:10A95000782343878287C28702464032118451841C
:10A960009184C183918000F02DF810BD500D00201E
:10A9700000FC0008AA550000F0B58C460025102602
:10A98000052109078E620E4C08E067467F5DE7608F
:10A99000A768FF07FCD0E7681F706D1C8542F4DBD9
:10A9A0000020074606E0E760A568ED07FCD0E568F3
:10A9B0001D54401C9042F6D38E610020F0BD000073
:10A9C0000030014070B572B60124074DA402214643
:10A9D0002846FBF703F9002804D0224603492846FD
:10A9E000FBF7A0F962B670BD00FC0008500D002016
:10A9F000F0B50025102605279C463F070B46BE6292
:10AA00000C4C06E0595DE160A168C907FCD0E16823
:10AA10006D1C8542F6DB002007E06146095CE160C1
:10AA2000A168C907FCD0E168401C9042F5D3BE6123
:10AA30000020F0BD003001400000010203040005C9
:10AA4000405C0000A05C0400C06C0800805C040056
:10AA5000E03F1E00E07D1E0007A9022570889B884C
:10AA60000A001600010006000100020087008D00A8
:10AA70002D001A3152001A339A001A351D011A3767
:10AA80006B003B31BE003B335E013B3596023B37EA
:10AA9000000099599959EB518F421E45142E0080A0
:10AAA000EB51F5283333E13A703DE13AC235852B5D
:10AAB000C2353333C235C235AE47E13A5138A330DF
:10AAC00051380000000000000000010203040607E6
:10AAD0000809030406080C101820300000000001CB
:10AAE0000203040004AB0008000000202401000061
:10AAF0000C9B000828AC00082401002074190000F9
:10AB00001C9B000800000000000000000000000086
:10AB1000070400091E0805400826091040085608C9
:10AB2000054008261D040008BE1D040008BED8BC50
:10AB300040100800010000000000C84200000000B2
:10AB40000000000000000000000000000000000005
:10AB500000000000000000000000000000000000F5
:10AB600000000000000000000000000000000000E5
:10AB700000005C1200000000000000000000000067
:10AB800000000000000000000000000000000000C5
:10AB900000000000000000000000000000000000B5
:10ABA00000000000000000000000000000000000A5
:10ABB0000000000000000000000000000000000095
:10ABC00000000000020204000909010200810000E7
:10ABD0000000000001000000000000000000000074
:10ABE0000000000000000000000000000000000065
:10ABF0000000000000000000000000000000000055
:10AC00000000000000000000000000000000000044
:10AC10000000000000000000000000000000000034
:08AC200000002000000000000C
:04000005080050C1DE
:00000001FF
